:020000040000FA
:020000000528D1
:0800080005282320051D3829FD
:1000100025104430AC004930AD00C2308720043098
:10002000AC004B30AD0096308720051D15283030D0
:10003000A00AA400051917286820A40B1A28061680
:100040008D2006121528831203138701860183125F
:10005000031700309E009F008316031300308700B3
:100060002F30860081131515831203179501831213
:100070000313682000308600A4012408482087006C
:100080005E20A40A0A302402031D3D2886170800BA
:10009000A9008A01290882073034383438343834CA
:1000A000083401340634083402340C34A9008A01BF
:1000B000290882078034C0349434D434000000000E
:1000C000000006170000000000000613682008006A
:1000D0000130A2001030A300A20B6F28A30B6C28E4
:1000E00008000430A40086128316031386128312BC
:1000F0000313682083160313861683120313A00AC2
:10010000861E7F28A40B73282008A1000800870002
:1001100086135E208617B001962825140621B001AB
:100120000430AC003030AD00051D942871200F2143
:10013000A201A20A2E0822060319A201A10B9928E6
:10014000A2080319A7280F210F21A203A0280F211D
:10015000AA000F21AD002A08AC000F212E08031DB4
:10016000BF28B00803190800B003B00331303007CE
:1001700084000008AC00840A0008AD00AD282E08F9
:10018000013C031DD6280F21AA000F21AB003130FE
:10019000300784002C088000840A2D088000B00AF3
:1001A000B00A2A08AC002B08AD0096282808143C99
:1001B000031DE628A801A70A2708043C0319002903
:1001C00027085620870086135E208617A808031D7F
:1001D000ED2820302E020319AD28A80A251CFB2883
:1001E000031061302E02031CFB287B302E02031803
:1001F000FB282030AE0225102E0887005E20AD2897
:10020000051D0029051902290621E628A701A801D4
:100210000130870086135E208617682008002C0CAA
:100220001F39831203178F0003132D0DA4002C0C0C
:10023000240C03178D0083168C170C14000000008B
:1002400083120C080313AE0003170E080313AF004C
:100250002C1B2F292C177F30AE052E0808002E0DE1
:100260002F0DAE00AD0A2C13AD1BAC0AAD13080068
:0E027000A00171200F39413E87005E20382921
:10046000192518251C252125252529052F053105A8
:10047000350539053B053F0541054305450547055C
:1004800049054B054D054F055105530555055705C4
:100490005905DB008A2E0125E5020A370A380A3998
:1004A000CA3B4B0081258501CB05CB098B0E8125ED
:1004B000A800CB1881253401CB1CCB1D810543013D
:1004C0000B268B2A8105DB028B330B36CB384B3A5C
:1004D0004B3C82257F068100CC0101268800CC069A
:1004E000012692000C0B01069A00CC0E0126A200F8
:1004F000CC1302062A06AD018C170C1A8C1C0306BD
:10050000432646064B018C27CC2A02265926DD01BC
:10051000CC2FCC330C37030673067626FA004D0138
:10052000840688068E26912696010D0D0D0E8D0FE0
:100530008226A2262601CD14CD158226AD262F01B6
:10054000CD18CD198226B726B901CD1ECD20CD21DB
:100550008426C906CE06D42659018D2E0D33812658
:100560006D018D38CD3A8206FA067C010D3F0E00F2
:1005700001278300CE0303270B070E271106CE0D9C
:10058000CE0E0E138E154E178E190E1C4E1ECE203B
:100590000E23CE254E280E2756075E0760076527D7
:1005A000680770077607FC27810788278E0793273F
:1005B00097279D008F128207A9073001CF19CF1A04
:1005C0008127B7010F21CF23CF258427D007D70755
:1005D000E0276501CF344F368227EF07F6004F3F03
:1005E000022805288701D004D005D0060108930011
:1005F000900A04281D28232827282D039018D01A94
:10060000501D501F9021D02303084C284F28D4019F
:10061000502E1030903102086808ED01903A903C5D
:10062000903E822880280201D10611088328940870
:100630009A089C025110D112D115D117D1198208F4
:10064000B908BB00D11F81284403112691279128A6
:10065000D12B112E112F8408E008E428E808ED03BF
:100660005139D13CD13F92025205D20612080609F7
:1006700013091509170919091B091D0152149216AE
:1006800004093029342939093D015220D2220309B5
:100690004A294E295402122DD22FD2341237012961
:1006A000F302D23B923D923FD302D30484298D2999
:1006B000902994091701130D13128109A8015317EA
:1006C0005318531B8229BA09C001D323D325D32839
:1006D0008429DB09E029E509EE02533BD33DD40030
:1006E000D4031407010A1301940B940D022A1D2A46
:1006F0009F001412010AB000D41A020A392A4201DA
:10070000D424D425030A4F2A530AD501542ED42FBA
:100710005431010AE903543654375439D43B943DDB
:10072000543F5501822A862A0D01D508150A840AEC
:100730009A2A9C2A9F0AA3001513820AAA0A2F014B
:10074000D519151C810A3C0115209521842AC52A3A
:10075000C72ACC2A4E01952A552D830AE02AE22A7F
:1007600064025533953415369538842AF30AF62AEF
:10077000F80A7B01953F9601080B050B090B0D2B21
:10078000140B190B1F2B272B2C019619961C020BEF
:10079000422B4901D6279629010B5701962F9630F7
:1007A000020B632B6401D6331638032B730B770BC4
:1007B000F902563E17005702D705D707840B940B52
:1007C000960B9B0B9F01971397155718832BB40B10
:1007D000B82B3B01571F5720812B42035723572526
:1007E0001728972B572DD731820BEA0BEC011737BF
:1007F0009739973B832BF90B7E0C0302580358055E
:1008000098061808032C130C1A2CA0015811D812A2
:10081000D814020C2E0C3001181D1820082C4A2C5C
:100820004C2C4E2C520C562C5A2C5D0C6102583319
:10083000D834D8361839022C760CFD019900D9012C
:100840009903832C892C8B2C8D02D9079909D90AFD
:10085000190CD90D840C9E0CA10CA82C2B01191875
:10086000991D820CC90CCC021927D928192B992C57
:10087000192E822CDF2C630199335935850CED0C30
:10088000EF2CF10CF70CFB011A00DA011A03022D10
:10089000090D0D039A07DA099A0C5A13DA16DA18B9
:1008A000022D3A2DC1015A249A25DA26022D4F0D28
:1008B00055015A2B5A2C022D5A2D5E035A305A32AA
:1008C0005A35DA371A3C5B00812D02015B035B0568
:1008D000872D920D9A2D9D0DA12DA42DAC0D3301C8
:1008E0001B1D1B1E822DC00DC2011B221B231B249E
:1008F000822DCB2D4C015B271B28810D52011B2C17
:100900009B2E832DE02DE52DE9005B37822DF92DFF
:10091000FB01DC009C021C04022E0B0E10035C0C7D
:100920005C0D1C0F5C12DC159C17030E340E360E8A
:1009300038021C1D1C1E5C22DC24052E4B0E502E82
:10094000540E590EDE011C311C331C36022E6F2E44
:1009500072019C3A1C3C022EFE2E06015D065D08CB
:10096000842E952E970E9C0E9E019D111D139D1495
:10097000882EAC2EB02EB22EB52EB72EBC2EBF2E8A
:10098000C400DD24830ECC2ED30E59015D305D31C1
:10099000832EE42EE90E6C025D371D391D3B1D3D93
:1009A000020F022F85005E050F0F100F142F190F75
:1009B0001F0F232F272F2C2F320F3C0F402F430FB9
:1009C000490F4F2F532F58011E2F5E31022F692FD1
:1009D000ED015E3ADE3BDE3C020F7B0F7E019F01A4
:1009E0005F04822F8A2F0F015F0A1F0C820F9A2F3C
:1009F0001E055F115F12DF139F159F165F195F1AA7
:100A00009F1B9F1D5F20820FC40FC8071F251F2635
:100A1000DF27DF285F2A1F2CDF2D1F2F1F30DF313C
:100A20001F335F349F355F379F39830FF50FF80F02
:100A3000FC00482CA00046258030A000850EA000B8
:100A4000853280000921A0008A018000843CA0003A
:100A5000051C800049298122141081040100012411
:100A60006500012258108104010001225F108103FA
:100A70006C000104090001047810010372000124D4
:100A80002E0001037A0001237B0001236400012270
:100A9000530081034C0081042B00812404000104D5
:100AA0007D008104060081025B00010262000104F6
:100AB00064008102600001037D00C5224710D63228
:100AC000F239E9376E10311730188030763A6137D5
:100AD000F3356917EE32F417E53267004621490015
:100AE000C32441008124C039E832F23466338000E7
:100AF0004920D3326339653AA0296539F634E332A7
:100B000080004920F037EC34E33280004426A00016
:100B10008823A000092880004426A0000514A00016
:100B20000839A000462D80004426A0000711A034FB
:100B30006E10EF3A72108122590001047810F730DC
:100B4000731081022810E23CA0004426A000462D2C
:100B50008024A0000602A033653AA000882DA037AB
:100B6000753A8024A0000634802420346132203A73
:100B70006F108000042D80000834A000C73EA0360E
:100B80006510F43720000104781081232A106137A2
:100B900064104910010362004910F7307310E23A03
:100BA000F33CA000C43BA0306E0001225B31651015
:100BB000613AA0306E004910F73073108124631041
:100BC0006131EF3A74100104021081225900CD30D6
:100BD000F235653A693767004F386539613AE93768
:100BE000EE3980296136E539002369376137E33210
:100BF000802661377533E131F43AF234EE33002B5D
:100C00005000E832613280327838EC37F3346F3795
:100C100000347932F2307536E9310036E933683A1A
:100C2000EE34EE330036EF31EB326400ED32653AEC
:100C3000693767006F33E634E3320038EF34F33757
:100C4000EE34EE338039F7306C36EF3B6532803B63
:100C5000693A6800611081222400010468000104DF
:100C6000E813731081221F006110012313108122E9
:100C70001A00611081221A107434613A2032E9326C
:100C8000641081040100ED3A723265390031753922
:100C9000673661397900F237623165397900E131BF
:100CA000E334E4326E3A6136EC3C8039EF36653439
:100CB000EF3B80004501A000091880000918803032
:100CC000A000C7242031F232E135E4377737803095
:100CD000A000C702A030743AE1316B00611001241A
:100CE000491001043900613661396D00EC37E33594
:100CF000E437773700336939651070396F3AE53179
:100D0000F4346F3780008505A039F939F4326D006D
:100D10006137A030E3316932653774006137A00074
:100D2000C4358030A0004539A0000913803020333D
:100D30006939650081021000611001027F0061378E
:100D4000A000050C8030F339E13A6C3A8030F2397A
:100D50006F378000CA02800008078000450D8000C0
:100D6000072F800008070038653AA000CA028000FB
:100D7000450D80000815A000450D80000815A00055
:100D8000450D8000450D8000450DA000C43BA0002E
:100D9000C71C80307239E539F4326400613870392B
:100DA00065346537E4326400E9367039E9396F3704
:100DB00065320035E134EC326400E13920396536C2
:100DC000613A6532203A6F10812440006937A000F3
:100DD000C711A0376610010402108030741081041E
:100DE0004800613AF430E335653280306D31F539D1
:100DF000E832640081223000E23474008122300045
:100E0000E234743A653780008519A0000839800003
:100E1000851DA000C43D003175397900E536E2300A
:100E2000EC3600346F366410EC30733A2039693A8E
:100E3000E53920336F39002132218036E939F33426
:100E40006F37AD31F234F434E3306C00733AF23082
:100E5000F432E734630067366F31613600346F3641
:100E6000E939F4346300ED30F235653A69376700EB
:100E7000653B6F36F634EE330038F237E131F43447
:100E8000F632803979376539E73463006537F432F3
:100E90007238F234F3320039E530EC16F434ED32C6
:100EA0008031EF36F032F434F434F63280346E337D
:100EB000F230733AF23A633A75396500D227490045
:100EC0006132F6306E3AE1336500ED307439693CD9
:100ED00080316F36EC30E237F230F4346F37730024
:100EE0006937693AE930F434F6327300E536F037A1
:100EF000F732F236653774006937E3326E3A693B90
:100F0000E53900326536693B65396131EC32730091
:100F1000F4326334EE37EC37E734E5398031E830CA
:100F20006E3765367300F030F230E434E7368039DE
:100F3000E330EC30E234EC34F43C8030E331EF3A2F
:100F40006E3A61316936693A790081223E10810238
:100F50004B000122DB00C805A00045168122590084
:100F60000122DB00C8050031F53C8033653A800082
:100F7000083CA000C606A000C603A0346E3A6F105D
:100F800001030B00E330F4316810E634F2328032B2
:100F90007838EC37E4328039E83A7410E437773740
:100FA0008036613265100124581081226100E330DF
:100FB000F5396532A000482C203A6F10812261007B
:100FC000E330F5396532A00005088000C60CA000AA
:100FD000482C8031E832E33580307532693A800040
:100FE000491AA00049206636EF3772008122691045
:100FF0008124C0346E3B6537F437F23C80000536FF
:10100000A0346E108124C000890E80004539800014
:10101000071E8000853C8000C53E8000C53EA000C4
:10102000493401240500810335006F39E9336937FC
:10103000613A693767106639EF360031F232E135CF
:101040002033EC3A69328031EF37EC306E3A80363B
:10105000693765396136A03769360031EC32E131E4
:101060006800E83C6439EF3365370038EC3AF43710
:10107000EE34F5368031F930EE34E43280316836C2
:101080006F3969376500EE347439EF336537003BEB
:1010900061376132E93A6D00E8306410F43780312D
:1010A000EF3A6C3220376F3A803BE13920376F3AA4
:1010B000A03062366510F4378036791081247800CC
:1010C0006110812478000104E813731081247800F2
:1010D0000104E8137310812478008124C000C43116
:1010E0002031F5346C32693767006339E139E83211
:1010F0006400F336E139E8326400E23A6D38653273
:101100008000C7268000093B2038EF39F332F339DD
:10111000E9376E106F33A00045390032E5306400C6
:10112000E432E332E1396532003265386139F43650
:101130006537740001027300E23A6936E434EE3335
:101140000032E5397439EF3C653280306E376934EE
:101150006936613A6532003AF230733465320032F2
:10116000E136E13365320032E5366F36E939E8328F
:101170006400E4346700E23A6C36E437FA32800007
:10118000860FA030A00049048000C610A0000933DB
:10119000A000492081041500F037F73272000102E7
:1011A0006D00E434733AF234E23AF4346F37003AC3
:1011B0006539ED34EE306C008104380081223E0048
:1011C000E732EE32F2306C00E434733AF234633AD0
:1011D0000039E533E937EE306C00E434F634F334AB
:1011E0006F37613680316F37F430ED34EE30F434E0
:1011F0006F370032E939F43A72316137E332003245
:10120000E939F23A703AE9376E00F43A72317536DC
:101210006537E3328039F437F236803B613B650055
:101220007334EF316B0001032300812239008123E5
:101230001B0001240B0081226E0001032310010416
:101240005610E23AF23CA030A000C609A000450DBD
:101250008034EE33E539F4326400643961376B0071
:10126000653B6136F530F4328030F231E834F432E7
:10127000633A8030F339E5397300E432E634EE3214
:101280008032F832E33AF434F63280366137E133B3
:1012900069376700653C70366F3265320032E93974
:1012A0006138F0326139653280336F3AA039F437F2
:1012B000EC326E006239EF356510E43777378033F2
:1012C0006F3AA031EC37E7336532A000C43BA00091
:1012D000053B80327838EC37E4326400E23A72370A
:1012E0006532A037753A8000C734A000092A8033E0
:1012F0006F3AA0346E00E6326C36A0346E00E737E9
:101300007410733AF5316B1069378031EC37E7337D
:1013100065320032E136E13365320033E933683A51
:101320008039E33A6633EC320032F5326C006239D0
:10133000E13B6C006F37A039F539F034E3346F3797
:10134000A037661081234D00E637721001031100AB
:10135000E73774106937A030A000062B8000862E76
:101360008000862EA000C43BA00008348000862E9A
:10137000A000890080336F3AA0000438A0346E00CA
:1013800001030410E7327410EF3A74106F338000D9
:10139000042FA00009288000083CA0000631A0000E
:1013A000092880000834A0000438A000483DA000AF
:1013B0008704A000890E80336F3A2036EF3974001D
:1013C000E7377410F23762316532803BE139A000B3
:1013D000C63F20317910611081247800F7307310F6
:1013E00081223510E23CA030A000051180336F3A15
:1013F0002032F23AEE3580336F3AA000880DA0001B
:10140000053880336F3AA0004539A000443A800087
:10141000C61EA039EF3665108122720081020510C8
:101420006110810374000103761081220700EE32FF
:10143000F43B6F396B0067396932003461328039AF
:101440007533E632F2326400E8306410F43720314C
:10145000651001244310F437A000492081030200E5
:101460000102DA00C52EA00009068000C42D010388
:10147000370001047810F730731001237F10E23C2D
:10148000A00007138030A0000713A000C63FA000F3
:10149000483A0034693A80397439F5316B00E837DD
:1014A0007338693A613680225200E5366539E73291
:1014B000EE317910F237EF3600386137E931003418
:1014C000E530723A00347938EF33EC3CE332ED34F6
:1014D00063006937203AE8320033EC3C003A653962
:1014E000ED34F4328031EF316B39EF3063348039D1
:1014F000F034E4327200E232653AEC328031F23498
:10150000E335653A003661327931F53380346E3B2C
:10151000E539F434E730F4346F3780302038F2376F
:10152000E2328035E53C7300E131E332F339A0313A
:1015300061396400EB346C360032F23777370038AB
:10154000EF34F3376E00F430F3327200810317107A
:1015500001046800E7376C33203161366C00E230FB
:10156000F332E2306C360036E13AEE31E8326400B4
:10157000733A6139F432640081231F108103120031
:10158000EC3467347400F634E53B80004437803631
:10159000653AE537F234F4328000870E80397439C9
:1015A000E13C20317536EC32740081032D10ED3CA6
:1015B000A000470A80008938A000492081220E003F
:1015C000EC37733A8030F4328000043B8036E134EB
:1015D0006C0070346F3765007338F234EE35EC32DE
:1015E0007200C321542B0032F5397400E434723A8E
:1015F0008039EF37740081221A1001241D008122E6
:1016000072100122740001244900C139F034F2340F
:101610006E00D43CEC32EE376C007336E532F034B9
:10162000EE3320386936EC39003B693AE1366937E8
:1016300073006137F434E2346F3AE9317300ED3A04
:10164000F331EC3220396536613C6137F439803949
:101650006532613A693BE53980306E3AE937F834F2
:10166000E4306E3A730081033C10E63772100124B7
:10167000740081033C10E63772100124F4137310D8
:1016800001244900012271106F37A0000801A00059
:10169000C52C8000C438A000C43BA00008348036AC
:1016A0006537F4306C00EE32723BEF3A7300812400
:1016B000D230A000CA02A0346E1081045000010292
:1016C0007F0081021800ED3C80000834A7398000BB
:1016D000492001034F106F33A03679108124780020
:1016E000ED3CA000493C803679108124780001242B
:1016F00074008124C000890E003BE131F53A6D0091
:10170000ED306737653AE9318033F230F634F43042
:10171000F4346F376136003AE832F2366136003819
:10172000EF39693AF2376E0081242D0001245210FE
:10173000733A6F396D008123581001232F008123E4
:10174000581001232F108122771081244B00012390
:1017500024100123730081233010F33C733AE536E3
:1017600080004812A00007330039EF3AF4327200CB
:1017700062396932E7320038F237F83C8000472C92
:101780008000091C8000073DA00087238039F430C9
:1017900070366539003861386539A031EC34700035
:1017A000F23A62316539A032F230F3327200F0322F
:1017B000EE3169360038F2346E3A6539A03161395C
:1017C00074396932E7320028EF39F416693A203764
:1017D0006F3A650081236D0081230A00E131F43402
:1017E000EE33A03A70006F33663669376500E43730
:1017F000773780376633AD39693A6500E936F037B7
:10180000723A613774007539E7326E3A8037723256
:1018100065396532003A6F366400E139EB326400B5
:10182000F7306E3A653280004920E3376D38613712
:10183000F91373008124C0316F39F037F230F4327C
:10184000803775398037F834E43280397536E630C0
:10185000F432803168366F39693265000104500016
:101860000104501061376410ED30E432A03474107C
:10187000812261000104311001040210812259000B
:1018800001051510611001243B106F37A0000801FD
:10189000A000C52C0032EF338031613A0034E136CC
:1018A000733A653980336539E2346C00F030F230D8
:1018B000EB32653A00346F39F33200386139F23770
:1018C00074006334693763346936EC300038E837C4
:1018D000EE320038F2346E3A653900376F3A6531CE
:1018E000EF376B00E3376D38753A65390038EF3400
:1018F000F337EE32641001227700E8346734A03702
:101900006E00F0376F388036613775396500733493
:101910002A3A8000C50F8000493C8000480B803285
:10192000AD36E1346C00482A54280024D4264C00FB
:10193000D421D0174928002BCF245000F230E234B4
:101940006400F331E834FA377034F232EE34630075
:10195000F039F931E837003265396137E732640030
:10196000ED3CA000493C20396137A037753AA037DB
:101970006610812272000102DA00C819A000492015
:101980008122721001043E106F33A0367910812439
:101990007800F2320103400001034000F232E634E5
:1019A0006C360039E531E830F2336500F03AF23355
:1019B00065006336E5306E00F232EC376132003993
:1019C00065366138F3328030743AE1316B00F232BF
:1019D000F037723A8036E5366F0001034F00F4307D
:1019E000EE358039F430E234EC34FA327200F232FF
:1019F000E131F4377200F232F332723BEF347200AD
:101A0000F23A733465328039653774006439693B62
:101A100065378039E530EC32640001027000E4344F
:101A200061397234E53000326538F232F339E93722
:101A30006E007338EC347410F032F2396F3761365F
:101A4000693A7910E434F337723265398039633496
:101A5000693D6F3868396537E930803661366139FC
:101A6000E9308039EC32653869376710F334E33593
:101A7000EE32F3398030A000C736A0004628A0001F
:101A800009218030A0004705A0004628A000C922F7
:101A90008039EE377700F23069378000443780397B
:101AA0006F104910E33775366400F437800047291A
:101AB0008000092180000728A00088108000483A93
:101AC00080367910E13A6E3A80367910EE32E93399
:101AD00068316F3980367910E337F53969378036E8
:101AE0007910ED3774346539A0346E10EC3077001E
:101AF00061106639E9326E32A0376610ED34EE328D
:101B0000800008348000083CA000462F8000083C7C
:101B1000A00046368000083CA0004636A0306E3259
:101B2000A000463C8000492001032B10ED30EE3030
:101B3000E73272008124C021C52780004920432359
:101B40004F008124C021D427800049200123441064
:101B5000E434F232633A6F39800049207039E53954
:101B60006932653774008124C0008434A037661060
:101B70000122630001046800F337ED32E237E43CF0
:101B80008036650001245D0001245D0001046800C9
:101B9000ED3CA000C50F80248000483A80366500E7
:101BA000012474000124741081246E1001247A0031
:101BB0000104E813731001241600ED3CA000480B4B
:101BC00080376E108124C000491180008704A00076
:101BD000890E803074108124C000490C8000C83701
:101BE000A000C63FA000882DA000C43BA030A000EC
:101BF00049078000042980000429A0306E32A0002B
:101C0000842B003AF232EE316800E330EE306C00A3
:101C1000F43A6E3765368039EF366510812344001B
:101C2000F337ED32A000453920336F39A000872A01
:101C30008000870E0034E136ED327200E230F3327C
:101C4000E2306C362031613A80366F37EB327910F2
:101C50007739653763348039E837F6326C00F03411
:101C6000F43168336F396B008124220081041D0038
:101C70008124180001027300733A6F39E133651053
:101C8000E630E334EC34F43C803B61396534EF3AC0
:101C9000F332003875310031E139E53665377400CB
:101CA000E2307434F237EF368000C9392039EF372B
:101CB0006D00E330E632F432F23461000122631049
:101CC00001031600E8346734F7307900F030F2355C
:101CD00069376710EC377400733AF232653A80392D
:101CE000F0346C360036E5306B00733A6F366500C1
:101CF000F437EF35A0376633A000C43B8000C83707
:101D0000A0004914A0000728A00088108000072820
:101D1000A0008810A0008623003A6F39EE30E43727
:101D200000347539F234E330EE328000043B803405
:101D3000EE33E539F4326400613A65006334EF351F
:101D40006532A0376E00F33BE53270006336E53054
:101D50006E00F037EC3473340037F531EC32613912
:101D60008033E13980397539E732800084360038B4
:101D7000EE32F536613AE9318039F030F23500382B
:101D8000F232E334F3346F378031F23CEF336537AE
:101D9000E931003AE83220008124C0004731A00038
:101DA0008704A000890E80004920812362108102EF
:101DB0002F008124C0008627A0008704A000890E80
:101DC000800009218000483F800049206F33E634BD
:101DD000E332803B6F396B00E837ED3280004920F9
:101DE000D33A6E008124C026EF376E00CA3AF03431
:101DF000F43272006110F33AF03272376F3B6110C7
:101E000001226B008124C000890E80000834A739AC
:101E1000A0008439003AE832F232A03BE1392000D8
:101E2000E132F230F4377200F33A7038F232F339BB
:101E30006F398031EF367039E539F3377200E933A5
:101E4000EE34F4327200613AEF36693D653900389C
:101E5000F237E332F3396F398036613769387536D6
:101E6000613A6F390038EF39693AE937EE34EE33C9
:101E70002032653BE9316500E937EE34FA32720011
:101E8000E730F335653A8037F83CE732EE30F43727
:101E90007200F430EE3520346F36E4327200F232E4
:101EA000F032613A65390038F237F432633A6F390B
:101EB0000032E537E437F234FA32720074346937AD
:101EC000EB34EE330031F2306937733A6F39ED3469
:101ED000EE33003A6839EF3A673480008704A03661
:101EE0006932643665106F33003A653AF230003A71
:101EF000F234003269007439E9326400613AF43234
:101F00006D38F432640081046C10F437A000870B44
:101F100080008519003AF234E73365396532803044
:101F2000633A693B613A653280396539F63272004D
:101F3000012271007537EC307733753680346C369A
:101F4000E533613680316139003AF23AE3350038E1
:101F5000E931EB3A7000F6306E00F335613A6531E5
:101F6000EF3072328029552B0031E9356500E234BB
:101F7000E33C63366500ED37F437F231F931EC328A
:101F80008029E533F7307900F7307310812376002C
:101F900001234A00E3377700F034E7326F37003926
:101FA000613A8036EF37F33200336539F23274002C
:101FB000EC34FA3072328033EF307400E230740067
:101FC000F2306231693A0031E53072006639EF3340
:101FD0000036E9376E00E737703465398039F13AF9
:101FE0006939F2326C0081230A007739693A650059
:101FF00070396538613965007039E53965377400C5
:02400E00D430AC
:00000001FF
